:1000000012C0189518951895189518951895189563
:100010001895189518951895189518951895189578
:100020001895189518958FE58DBFC0E4E6E24E2E21
:1000300084E08EBFD4E0F4E05F2EEEEFF3E0A0E6C4
:10004000B0E088278D933197E9F785E089B980E0A2
:1000500080BD88E18AB9662481E080939D00B89ACA
:100060008F9A8D9A8E9A80E080939C00C09882E34C
:1000700090E00BD3C09A82E390E007D3C09882E36C
:1000800090E003D3C09A82E390E0FFD2C0989798A3
:1000900096989598A0E6B0E022D344E650E060E060
:1000A00070E0A0E6B0E00D911D912D913C9122D31E
:1000B00014F009F004C0A0E6B0E0A8D2EECF8E9A0A
:1000C0008D9A9598ACE9B0E098E08D91983018F44D
:1000D000392F992702C038E098508795969808F4F0
:1000E000969A00000000959AEF93FF93E2E0F0E00B
:1000F000C3D2FF91EF919598EF93FF93E2E0F0E088
:10010000BBD2FF91EF913A9541F79923F1F68E9A80
:100110008D9A9598ACE9B0E098E08D91983018F4FC
:10012000392F992702C038E098508795969808F49F
:10013000969A00000000959AEF93FF93E2E0F0E0BA
:100140009BD2FF91EF919598EF93FF93E2E0F0E05F
:1001500093D2FF91EF913A9541F79923F1F68E9A58
:100160008D9A9598ACE9B0E098E08D91983018F4AC
:10017000392F992702C038E098508795969808F44F
:10018000969A00000000959AEF93FF93E2E0F0E06A
:1001900073D2FF91EF919598EF93FF93E2E0F0E037
:1001A0006BD2FF91EF913A9541F79923F1F68E9A30
:1001B0008D9A9598ACE9B0E098E08D91983018F45C
:1001C000392F992702C038E098508795969808F4FF
:1001D000969A00000000959AEF93FF93E2E0F0E01A
:1001E0004BD2FF91EF919598EF93FF93E2E0F0E00F
:1001F00043D2FF91EF913A9541F79923F1F6979AFF
:1002000000000000000000009798000000008E9A97
:100210008D9A9598ACE9B0E098E08D91983018F4FB
:10022000392F992702C038E098508795969808F49E
:10023000969A00000000959AEF93FF93E2E0F0E0B9
:100240001BD2FF91EF919598EF93FF93E2E0F0E0DE
:1002500013D2FF91EF913A9541F79923F1F68E9AD7
:100260008D9A9598ACE9B0E098E08D91983018F4AB
:10027000392F992702C038E098508795969808F44E
:10028000969A00000000959AEF93FF93E2E0F0E069
:10029000F3D1FF91EF919598EF93FF93E2E0F0E0B7
:1002A000EBD1FF91EF913A9541F79923F1F68E9AB0
:1002B0008D9A9598ACE9B0E098E08D91983018F45B
:1002C000392F992702C038E098508795969808F4FE
:1002D000969A00000000959AEF93FF93E2E0F0E019
:1002E000CBD1FF91EF919598EF93FF93E2E0F0E08F
:1002F000C3D1FF91EF913A9541F79923F1F68E9A88
:100300008D9A9598ACE9B0E098E08D91983018F40A
:10031000392F992702C038E098508795969808F4AD
:10032000969A00000000959AEF93FF93E2E0F0E0C8
:10033000A3D1FF91EF919598EF93FF93E2E0F0E066
:100340009BD1FF91EF913A9541F79923F1F6979A56
:100350000000000000000000979800000000A4E6E4
:10036000B0E0E4E8F7E0B1D18E9A8D9A9598A4E6D2
:10037000B0E090E28D91983018F4392F992702C09F
:1003800038E098508795969808F4969A00000000F7
:10039000959AEF93FF93E2E0F0E06ED1FF91EF9139
:1003A0009598EF93FF93E2E0F0E066D1FF91EF9133
:1003B0003A9541F79923F1F68E9A8D9A9598ADE981
:1003C000B0E098E08D91983018F4392F992702C049
:1003D00038E098508795969808F4969A00000000A7
:1003E000959AEF93FF93E2E0F0E046D1FF91EF9111
:1003F0009598EF93FF93E2E0F0E03ED1FF91EF910B
:100400003A9541F79923F1F6979A00000000000011
:10041000000097980000000086E086B9379AAFD1B7
:10042000A8E7B0E03FE003D1A7D141E050E060E0B1
:1004300070E0A8E7B0E071D1BB27A0E10D911D915C
:100440002D913C9157D109F002C0C09A01C0C098CB
:1004500096D1A8E6B0E03FE0EAD08ED190D1A6EAEE
:10046000B0E03FE0E4D088D18AD1ACE8B0E03FE032
:10047000DED082D10000000000000000000000007B
:100480000000A8E6B0E049D1A4E6B0E00D931D93CA
:100490002D933D93A6EAB0E040D1A2EAB0E00D93DF
:1004A0001D932D933D93ACE8B0E037D1A8E8B0E0C0
:1004B0000D931D932D933D93A0E6B0E0E8E8F7E09F
:1004C00004D1A2EAB0E04D915D916D917C91A0E6DE
:1004D000B0E00D911D912D913C910CD114F009F0DB
:1004E00094C0A4E6B0E00D911D912D913C91A8E837
:1004F000B0E04D915D916D917C91F7D0A4E6B0E0B4
:100500000D931D932D933D938E9A8D9A9598A4E605
:10051000B0E090E28D91983018F4392F992702C0FD
:1005200038E098508795969808F4969A0000000055
:10053000959AEF93FF93E2E0F0E09ED0FF91EF9168
:100540009598EF93FF93E2E0F0E096D0FF91EF9162
:100550003A9541F79923F1F68E9A8D9A9598ADE9DF
:10056000B0E098E08D91983018F4392F992702C0A7
:1005700038E098508795969808F4969A0000000005
:10058000959AEF93FF93E2E0F0E076D0FF91EF9140
:100590009598EF93FF93E2E0F0E06ED0FF91EF913A
:1005A0003A9541F79923F1F6979A00000000000070
:1005B000000097980000000000000000000000000C
:1005C00081E087B971D0AEE9B0E08D939C9380E073
:1005D00087B96AD0A0EAB0E08D939C930000000038
:1005E000000000000000000032E0AEE9B0E03BD0C7
:1005F0000000000000000000000032E0A0EAB0E0CF
:1006000032D0A0E6B0E002D05CCF09CF0D911D91B1
:100610002D913C9181E0080F8827181F281F381F53
:100620003C932E931E930E930895AEE0B4E017D042
:100630008D3049F0883079F03323C9F38D933A95A2
:1006400063FE16D0F4CF63FC03C012D08AE010D052
:1006500088278C9308950CD011973395E8CF5F9B32
:10066000FECF8CB108958D9103D03A95E1F70895AE
:100670005D9BFECF8CB908953197F1F7089568948A
:1006800062F80895E89462F80895EF93FF93EE27D7
:10069000E82BE92B31F0EDECFAE03197F1F7019717
:1006A000D1F7FF91EF910895369A3699FECF369A99
:1006B0003699FECF84B195B10895C8953196002042
:1006C000089591E005C092E003C094E001C098E075
:1006D000F4DF0D929A95E1F7089582E001C084E07D
:1006E00099279D938A95E9F70895040F151F261FF2
:1006F000371F089504171507260737070895000FB9
:10070000111F221F331F08950095109520953095D5
:100710000F5F1F4F2F4F3F4F0895002711272227AC
:1007200033271DD08A3328F4803318F005D015D034
:10073000F9CF0EF4E9CF089580538F93402F512FB6
:10074000622F732FDCDFDBDFD0DFD9DF8F919927BA
:10075000080F191F291F391F08958D910895E894D6
:10076000FCDF8032E9F38B32D9F38930C9F38D3263
:1007700011F46894F2CF0895E89463F808956894AA
:0C07800063F8089500366E0101000000CF
:00000001FF
